:020000040000FA
:0800000000008A110A123029E8
:06000A0083120313981C91
:100010000B28181218168C1E0F281A0810280030EA
:10002000080083120313B901BA01BB01003039047F
:10003000031D2E283A08E83A031D22283B08033AFC
:1000400003192E28BA0A0319BB0A8A110A120520BD
:100050008A110A1283120313B900162839080800FE
:1000600083120313B80100303804031D40288A119D
:100070000A1205208A110A1283120313B8003328CA
:100080003808080083120313B600B5007F08B400D7
:10009000B701B61BB7033608632083120313B501FB
:1000A0003408B6006320080083120313B300803EB7
:1000B000763E031C5E283730B30760283030B30724
:1000C00033089F20080083120313B100310E0F394B
:1000D000B200F030B219B2040F30B20532088A1102
:1000E0000A1254208A110A120F30831203133105A9
:1000F000B2008A110A1254208A110A1208008312CF
:100100000313AF007F08AE007E08AD002D08FE008F
:100110002E08FF002F088A110A121D218A110A12C7
:1001200083120313B000300803199E2830089F2063
:1001300083120313AD0A0319AE0A8628080083123E
:100140000313AC00831203130C1EA22883120313A3
:100150002C08831203139900080019308316031327
:10016000990018151812071387178312981783160A
:100170000C128C1218138312181318168316981663
:100180000800FC20831203130C1DC2280421A500C3
:100190007F08A400831203130C1DCA280421A700A2
:1001A0007F08A600831203130C1DD2280421AB0084
:1001B000A9007F08A80024082802AA002508031C1B
:1001C000250FAB022A08FF002B088A110A124220D1
:1001D0008A110A120A308A110A129F208A110A1201
:1001E000831203132608A4002708A5002808A600E8
:1001F0002908A700D22808000130831203139000B9
:10020000053097000C1108008312031315088312A0
:100210000313A00083120313160883120313A10013
:10022000831203130C11831203132008A200210868
:10023000A3002208FF0023080800003A031924291C
:10024000803A03192B2900347E08840083137F1819
:100250008317000808007F088A007E0882000800D3
:060260008A110A12C128F8
:00000001FF
